:020000040000FA
:10000000850186018316073085008601831207303B
:100010009F002F2882076F340334763457341B3403
:100020005D347D3407347F345F343F3479346C344D
:1000300073347C343C346D343934013463343834B3
:1000400068343534313471343E341F34303419342B
:1000500078346B3461346534683410345434A3011B
:10006000A501A4016B207E2060209020051C45285E
:1000700005193628051C4528051D3A28A30A2130F4
:1000800023020318A3016B203628A4176B208518C0
:1000900047282330A500702087202130A50070203C
:1000A00001302307A2006020A20B5328A4012230B4
:1000B000A5007020752060206020602060202F281F
:1000C000FA30A000C830A10000000000A10B642895
:1000D000A00B6228080023080A20240486000800D8
:1000E00025080A202404860008006430A200851731
:1000F0009B2085139920A20B772808006430A2006A
:1001000085179D2085139920A20B80280800643054
:10011000A20005179B2005139920A20B892808002F
:100120006430A20005179D2005139920A20B922888
:10013000080050309E2808309E280430A00032303D
:10014000A10000000000A10BA128A00B9F2808001F
:02400E00103F61
:00000001FF
